:100000000DC023C022C021C020C01FC01EC01DC003
:100010001CC01BC0010A2A4B7A85FF0011241FBE99
:10002000CFE9CDBF20E0A0E6B0E001C01D92AA3725
:10003000B207E1F7E1E6F0E012828EEF80936F0005
:100040001682612C712C65D089C0DACF26EB33E0A3
:10005000019720F0F9013197F1F7FACF089588EE72
:1000600093E0F4CF81E687B986EC86B9369A089595
:10007000369A3699FECF85B10895EF92FF920F938D
:100080001F93CF93C82F8B0184E1E82E80E0F82ED8
:10009000CC2361F0F701849186BFC801D7DF16BE7B
:1000A000C801D4DFC801D2DFC150F2CFCF911F9178
:1000B0000F91FF90EF900895CF93DF93D82F64E1D5
:1000C00070E08AE0DADF84EF91E0C0DF8D2F64E634
:1000D00039D0CAE06C2F36D0892F68EC70E0CDDFC4
:1000E000BEDF8D2F6C2F2ED0D92F2CD0892F68EC0E
:1000F00070E0C3DFB4DF68EC70E08D2FBEDFAFDFF0
:1001000064E170E08AE0B9DF84EF91E0DF91CF91A4
:100110009DCF8FE384BBB89A81E08FBD83BF8FB53D
:1001200080688FBD97B328B3892F90E08095909514
:100130008B7F822B88BB96DF8CE291E087DF98DF94
:10014000BBDFFACF991B79E004C0991F961708F01E
:10015000961B881F7A95C9F780950895F894FFCF6C
:00000001FF
